:020000040000FA
:06000000653002303A28D1
:08000800A000030EA100831209
:1000100005191028831601178312B23081002B288E
:1000200083160113831203140B190310A80DA90DD5
:10003000AA0DAB0DAC0DAC16FF302C02031D2B2806
:10004000FA302B02031D2B2831152A08AF0029088E
:10005000AE002808AD008B100B11210E8300A00EFE
:04006000200E090065
:0C007400203084008001840A6030040207
:10008000031C3C281230B0008E218316FF23900001
:10009000831283160C308505870183128501870141
:1000A000073099000030831691009F008312C830FA
:1000B00083168100831231309000003083168C004B
:1000C000831210308B001E2281018E018F010B11D3
:1000D0008B100B108C018B177B2031197E20B30BFA
:1000E0007928031085190314B90DF030390203196A
:1000F00005211F226C2864003210080031110130E4
:10010000B70085148B132030370783169B001C140F
:100110001A088312A4001030370783169B001C14A2
:100120001A088312A300A6000230A6060030370783
:1001300083169B001C141A088312A200A70001302A
:10014000A7068B17321CAA2822090339A200A3098B
:10015000A409A50924082F02031DFF2823082E0245
:10016000031DD22822082D02031DFF28013037026B
:10017000031DBD283D143E14A32102303702031D88
:10018000C428BD143E14AB2103303702031DCB2815
:100190003D153E14B32104303702031DD228BD158E
:1001A0003E14BB2126082E02031DF72827082D0226
:1001B000031DFF2801303702031DE1283D103E14C6
:1001C000C32102303702031DE828BD103E14CB21A5
:1001D00003303702031DEF283D113E14D3210430B4
:1001E0003702031DF628BD113E14DB21FF285F08EE
:1001F000AB3C0319FF282E1AFF28FE28E321B70A7B
:10020000053037020318080082280130B600B30019
:10021000B400B500B70085018701B11308227B2027
:10022000B30B4029031085190314B90DF0303902BE
:1002300003196729B41F8501B41F8701B41F8510F6
:10024000B40B4029B50B40290230B500013037020C
:100250000319EC21023037020319F1210330370270
:100260000319FA2104303702031903223708B608AC
:100270000319B60003193E298514B603FA30B400F9
:10028000311D0F293111321C4A292D090339AD00C6
:10029000AE09AF092F1C0F298E018F010C1C0F29ED
:1002A0000C102E1E0F298B1320303707BB002F0890
:1002B000BA007B2110303707BB002E08BA007B2123
:1002C00000303707BB002D08BA007B218B170C22AA
:1002D00085018701B70AB60105303702031C0F29D3
:1002E0001E2208003E1C08003E101030BB003D08D6
:1002F000BA007B2108008B133A0883161C159A005C
:100300003B089B0055309D00AA309D009C14640062
:100310009C1887291C1183128B1708008316003044
:100320009B001C141A088312DF00831620309B00E8
:100330001C141A088312C1000130C11BC100C1087E
:100340000319C10008000712871640084107D000B2
:100350000F08D10008000512871540084107D20098
:100360000F08D30008000711851640084107D40084
:100370000F08D50008000710871440084107D60071
:100380000F08D70008008712071640084107D00061
:100390000F08D10008008711051640084107D20058
:1003A0000F08D30008008512071540084107D40044
:1003B0000F08D50008008710071440084107D60031
:1003C0000F08D7000800071205120711071087123F
:1003D00087118512871008003F0930398700BF0058
:1003E0000800380910398500B8003F09083987002E
:1003F000BF000800380920398500B8003F090439DA
:100400008700BF0008003F0903398700BF000800CC
:10041000B801BF01BF160800B801BF0101303702A3
:10042000031D132ABF1502303702031D182AB81600
:1004300003303702031D1D2ABF14080008005008AE
:100440004002031D292A51080F02031C292A071202
:10045000871252084002031D332A53080F02031C5F
:10046000332A0512871154084002031D3D2A5508FE
:100470000F02031C3D2A0711851256084002031D76
:10048000472A57080F02031C472A071087100C1C25
:1004900008000C10C00A851008000C1C6C280C10F9
:0E04A000C00B6C284108C000850187010800D0
:084000000100030005000100AE
:02400E00CC01E3
:10420000010078007A007C007E007B0079007F004E
:104210007D007A0078007E007C00FF00FF00FF0038
:104220000000F200F600FA00FE00F200F600FA00CC
:10423000FE00F200F600FA00FE00FF00FF00FF00A3
:10424000010005000500050005000900090009003E
:1042500009000D000D000D000D00FF00FF00FF0024
:10426000FF00FF00FF00FF00FF00FF00FF00FF0056
:10427000FF00FF00FF00FF00FF00FF00FF00FF0046
:10428000FF00FF00FF00FF00FF00FF00FF00FF0036
:10429000FF00FF00FF00FF00FF00FF00FF00FF0026
:1042A000FF00FF00FF00FF00FF00FF00FF00FF0016
:1042B000FF00FF00FF00FF00FF00FF00FF00FF0006
:1042C000FF00FF00FF00FF00FF00FF00FF00FF00F6
:1042D000FF00FF00FF00FF00FF00FF00FF00FF00E6
:1042E000FF00FF00FF00FF00FF00FF00FF00FF00D6
:1042F000FF00FF00FF00FF00FF00FF00FF00DD00E8
:00000001FF
